:084EDB0033302E3220202000AC
:10162600E4F5D975FF8075EF02751F21124C08AFDE
:101636001F124E3B43F6011248D8D2AF124CF71296
:101646004585124BE9124DCBEF6010124AE3123F6B
:101656001B3009F1C209120AA780EA1237F1900578
:10166600B5E07002A3E060329005B6E024FFF0908A
:1016760005B5E034FFF0E07002A3E0700B7BFF7A63
:101686004E79DBAF1F12416630180FE49005B5F0B6
:10169600A3F0A215B392151245851248ACEF70035C
:1016A6000217571243D0EF24FE602224FE60232443
:1016B600FC603D14606E14607B24FA605124F06077
:1016C60055241F600302174B1249538078124BAA08
:1016D600807390054EE07005740DF080347B017ABE
:1016E60005794E900684740DF07DFF124610802118
:1016F60090054EE0B40D04E4F080117B017A057983
:101706004E900684740DF07D011246108003121A65
:101716001B124585802F9005B57488F0A374B8F028
:10172600C2188021900531A3E0FAA3E0F5828A83EE
:101736007F01800E900531A3E0FAA3E0F5828A834B
:101746007FFF1224601248ACEF60030216A9121A3A
:10175600277B017A057998124880EF700302164BB1
:10176600C21B90059AE024FC607B14700302182EBD
:1017760024EFB40900400302187A90178E75F0031F
:10178600A4C58325F0C583730217A90217B30218EF
:101796007A02187A0217BA0217D702187A0217DFE6
:1017A6000217E5D215121A15D21B02187AC215D2E3
:1017B6001B02187A7B017A0579989005A8EBF0A3AD
:1017C600EAF0A3E9F012226C651F600302187A8022
:1017D60000AF1F124B4802187A124F0202187A12F3
:1017E6004F2102187A7B017A0579989005ABEBF0C8
:1017F600A3EAF0A3E9F0900003122285651F707436
:1018060030156C9005AB04F0A3EAF0A3E9F0900064
:1018160005122285FF900006122285FD9000041213
:101826002285FB123CFA80477B017A057998900560
:10183600ABEBF0A3EAF0A3E9F09000031222856572
:101846001F70313015299005AB04F0A3EAF0A3E927
:10185600F0900005122285FF900006122285FD9069
:101866000004122285FB123A7612492C124C41AF23
:101876001F124BCA2015030219BD90059AE0146089
:101886003624FA6074147003021969240660030290
:1018960019BD124DDD7B017A0579989005A8EBF00C
:1018A600A3EAF0A3E9F0900003122285F561124E37
:1018B600A8124EC70219BD124DDD7B017A05799833
:1018C6009005A8EBF0A3EAF0A3E9F090000312223A
:0918D60085F56112492C124EC780
:1018DF009005B1122405000186A09005B174FF1286
:0D18EF0023D2E4FBFAF9F8C31223BF40ED49
:1018FC000219B8124DDD7B017A0579989005AEEB93
:10190C00F0A3EAF0A3E9F0900003122285FF900007
:10191C0004122285FD900005122285FBC003900560
:10192C00AEE0FBA3E0FAA3E0F9900006122285904A
:0E193C0005E0F0D0031239C212492C124EC73A
:10194A009005B1122405000186A09005B174FF121A
:0D195A0023D2E4FBFAF9F8C31223BF40EDDD
:10196700804F124DDD7B017A0579989005AEEBF03B
:10197700A3EAF0A3E9F0900003122285FF90000488
:10198700122285FD900005122285FB122BEB1249CE
:041997002C124EC7F9
:10199B009005B1122405000186A09005B174FF12C9
:0D19AB0023D2E4FBFAF9F8C31223BF40ED8C
:1019B800124C41D21B201B03021757121A2712453B
:0119C8008599
:0319C900021757AB
:104D260075B980E4FF0FEFB414FB43B9C0E5B930A1
:054D3600E5FB75A90377
:014D3B002255
:104CC60075A41F75A5E0E4F5A675F2E77590FF7566
:094CD600D40875E10775E24222E1
:0A4EB30075A14075F801E4F5A22294
:104D3C00758922758E05758A5F758C5F758B4075CC
:064D4C008D407588502225
:0B4E920075CA3075CBF8D2CAD2AD2231
:104C0800124D26124CC6124EB3124D3C124E921241
:0E4C18004E48124C26124F27124DEE02463D1A
:1033AF0042042D00004203D800004203D30000C1A5
:0533BF0013C112C11151
:0A4EBD00C212C213E49003D7F022E2
:104A3600E490042DF0A3F09003D8F0A3F0A3F09037
:104A460003D3F0A3F09003CEF0A37440F0E49003F8
:034A5600D6F02275
:064F0900124EBD024A3603
:0D4E2E0075C19043E6019003D57401F02298
:104DDD0043C140E5C120E5FB124F09E49003D5F036
:014DED0022A3
:0A4EC70053C1BF9003D57401F0221F
:0D4E3B00AE07124E2E9003D2EEF0024F098A
:1049ED00E49006B0F0A3F0301202FF222013FDD2A6
:1049FD00129003D0E4F0A37410F090041BEFF0E4D8
:044A0D00A3F07F0192
:014A11002282
:1047550030120A9003D0E07002A3E070037F0022BC
:104765009003D1E024FFF09003D0E034FFF09004F3
:104775001CE0FE04F0741D2EF582E43404F583EF8D
:04478500F07F01229E
:0B4E9D00301207C212D213124ED122B5
:0A4ED100E5C120E5FBC2C4D2C522F2
:103F990090064FEBF0A3EAF0A3E9F09003D5E070A7
:103FA90002FF22900652E0FE6005D3941040037F81
:083FB90000221249EDEF604EF9
:103FC100E4900654F0900652E0FF900654E0FEC3E0
:103FD1009F502490064FE0FBA3E0FAA3E0F98E8204
:103FE100758300122285FF124755EF7002FF229060
:103FF1000654E004F080CEE49003D7F0124E9D9079
:0E4001000653E070032013FD9003D7E0FF226A
:03400F007FFF220E
:0E35DF00900685EBF0A3EAF0A3E9F0A3EDF06F
:1035ED00E4FFD390042EE0940090042DE0648094C9
:1035FD008050012253E6FE9003D3E0FEA3E024DACF
:10360D00F58274033EF583E0FF9003D3E475F0017A
:10361D00122393FCE5F064404C70069003D3F0A3A5
:10362D00F09003CFE004F070069003CEE004F0E4D8
:10363D00FE900688E0FDEEC39D5054EEC39F504FA3
:10364D009003D3E0FCA3E024DAF58274033CF58308
:10365D00E0FD900685E0FBA3E0FAA3E0F98E82750C
:10366D008300ED1222E69003D3E475F0011223934B
:10367D00FCE5F064404C70069003D3F0A3F090038A
:10368D00CFE004F070069003CEE004F00E80A2EEC1
:10369D00C39F50299003D3E475F001122393FCE5E9
:1036AD00F064404C70069003D3F0A3F09003CFE08C
:1036BD0004F070069003CEE004F00E80D290042E3C
:1036CD00E024FFF090042DE034FFF043E601900676
:0C36DD0088E0FEEFC39E50028002AF06A2
:0136E90022BE
:104CDF00D390042EE0940090042DE06480948040E3
:084CEF00047F0180027F002216
:031A1800022A504F
:102A5000C0E0C0F0C083C082C0D075D000C000C04C
:032A600006C007A6
:102A6300C21CE5C054FE1224362B3F082B3F0A2B11
:102A7300060C2B060E2BB8102BB8122B0C222B177F
:102A8300282B172A2B0C2C2B0C2E2AF9C02AB2C266
:102A93002A9DE02A9DE200002BC3C21190041BE093
:102AA300F5C2C2C5C2C490041A74FFF0022BC590CC
:102AB300041AE0FFB4FF1290041CE0F5C2C2C5C2C1
:102AC300C490041AE4F0022BC590041CE0FEEFC38B
:102AD3009E501790041AE0FF04F0741D2FF582E452
:102AE3003404F583E0F5C2022BC5D2C49003D7E4C6
:102AF300F0C213022BC59003D774FDF0D2C5C2C434
:102B0300022BC590041A74FFF0D211C2C4C2C1D201
:102B1300C5022BC5E5C260079003D2E0B5C20E9093
:102B230003CDE4F0C2C5C2C4D2C1022BC5C2C4C224
:102B3300C1301103022BBDC2C5022BC59003CDE0EA
:102B43007020E5C2F0E0FFC39003CFE09F7480F8EC
:102B53009003CEE06480985003124A369003CDE090
:102B630004F09003CFE024FFF09003CEE034FFF0B5
:102B73009003D8E0FEA3E024DAF58274033EF583E4
:102B8300E5C2F09003D8E475F001122393FEE5F05B
:102B930064404E70069003D8F0A3F09003CDE01488
:102BA300F0700E90042EE004F0700690042DE00403
:102BB300F0D2C1800DC2C4301108C211D2C5800247
:102BC300D21C301C1053C17F43C180C2C5C2C4C2D2
:072BD300C1C21CC213C2C005
:102BDA00D007D006D000D0D0D082D083D0F0D0E0B9
:012BEA0032B8
:054F0F00E5C15420FF84
:014F1400227A
:0E454000900663EBF0A3EAF0A3E9F0A3EDF020
:10454E00E4900668F0900663E0FBA3E0FAA3E0F9BE
:10455E00A3E0900652F0900667E0900653F0E4FF59
:10456E00123F99EFB4FF0D900668E0FE04F0EEC323
:06457E00940340D17E0011
:014584002214
:0B4880009006A1EBF0A3EAF0A3E9F022
:10488B007E007F007D101224629006A1E0FBA3E066
:10489B00FAA3E0F97D101235DFEF7002FF227F01E2
:0148AB0022EA
:104166009005F47422F0A3EFF0A37413F012226CFE
:104176009005F7F09000011222859005F8F0900066
:10418600021222859005F9F090000312228590050F
:10419600FAF09000041222859005FBF090000512BB
:1041A60022859005FCF09000061222859005FDF010
:1041B6007B017A0579F4E4900667F07D0A024540B2
:104B27009006897422F0A3EFF0A37403F0A374FF37
:104B3700F07B017A067989E4900667F07D040245E7
:014B4700402D
:104B480090068D7422F0A3EFF0A3741CF0A374FFF9
:104B5800F07B017A06798DE4900667F07D040245C2
:014B6800400C
:104BCA00E4900691F0A3EFF0A3740AF0A3EFF07B50
:0F4BDA00017A067991E4900667F07D0402454068
:074EFB0043C14053E6FE2213
:102EB300900612E0FFA3E0FCA3E0FDA3E0FBA3E088
:102EC300FAA3E0F99005EFE554F0E555A3F0900679
:062ED3001AE09005F1F089
:102ED9009005E9EFF0A3ECF0A3EDF0A3EBF0A3EA82
:042EE900F0A3E9F079
:102EED009005F27403F0A374E8F0E5C120E5FBD280
:102EFD00C1C2C4D2C5E4FF9006BBF030C0FDE5C031
:102F0D0054FE24407003022FB024FE602424E2609E
:102F1D000924FE600524E2022FB8C2C5EF6003024A
:102F2D002FBE9005E9E025E044A0F5C27F03022FF6
:102F3D00BEEFB4030A9005EAE0F5C27F058072EF9B
:102F4D00B4050B9005EAA3E0F5C27F068063EF643C
:102F5D0006703E9005F1E09005EC700FE0FBA3E4E8
:102F6D0075F0011223A9A9F0FA8008E0FBA3E0FA9D
:102F7D00A3E0F912226CF5C29005F0E024FFF09069
:102F8D0005EFE034FFF0E07002A3E070247F0780CE
:102F9D0020EFB40706D2C47F0980169006BB7405D6
:102FAD00F0800E9006BB7402F080069006BB740193
:102FBD00F0EFB40904C2C080369006BBE0FE640693
:102FCD006012EEB402169005F274FFF5F012239321
:102FDD0045F06008D2C5E49006BBF0FF9006BBE05B
:102FED006008C2C5D2C4C2C08005C2C0022F08E5A8
:042FFD00C120E5FB0F
:0130010022AC
:103002009005FEEFF0A3ECF0A3EDF0A3EBF0A3EA42
:04301200F0A3E9F04E
:103016009006067403F0A374E8F0E5C120E5FBD240
:10302600C1C2C4D2C5E4FF9006BBF030C0FDE5C006
:1030360054FE24C870030230F324AE607A24CA70AA
:10304600030230FB24FE603824E2600924FE60059A
:1030560024E2023103C2C5EF700F9005FEE025E0C1
:1030660044A0F5C27F03023109EF64016003023117
:10307600099005FEE025E044A1F5C27F040231096E
:10308600EFB4030A9005FFE0F5C27F058075EFB443
:10309600050B9005FFA3E0F5C27F068066EFB40638
:1030A60006D2C57F01805CEFB404047F0280549091
:1030B60006BB7405F0804C900601E0FBA3E475F0B6
:1030C600011223A9A9F0FAE5C21222D4900605E05E
:1030D60024FFF0900604E034FFF0E07002A3E070F5
:1030E600087F09C2C1D2C4801A7F0280169006BB2F
:1030F6007406F0800E9006BB7402F080069006BB44
:103106007401F0EFB40904C2C080369006BBE0FE3D
:1031160064066012EEB4021690060674FFF5F0120D
:10312600239345F06008D2C5E49006BBF0FF9006F5
:10313600BBE06008C2C5D2C4C2C08005C2C00230AE
:0631460031E5C120E5FBAC
:01314C002260
:1036EA00900612EFF0900615EBF0A3EAF0A3E9F0CA
:0836FA00900613ECF0A3EDF0C3
:10370200755600543FF557543F605CC3744095575B
:10371200FFE49556FE900618E0FCA3E0FDC39FEC83
:103722009E50068C548D5580048E548F55122EB3A4
:103732009006BBE060037F0222900614E02555F05C
:10374200900613E03554F090061AE0700B900616BE
:10375200E5548555F0122393C3900619E09555F070
:10376200900618E09554F0900618E0F554A3E0F5A1
:1037720055D3E5559400E55494004070E5559440C6
:10378200E55494005013122EB39006BBE060037F01
:103792000222E4F554F55580D8900612E0FFA3E02A
:1037A200FCA3E0FDA3E0FBA3E0FAA3E0F99005EFA0
:1037B200E4F07440122ECF9006BBE060037F022239
:1037C20074C02555F55574FF3554F554900614E030
:1037D2002440F0900613E03400F090061AE0709155
:0E37E20090061675F0401223930237737F0095
:0137F00022B6
:104D0F00900604E4F0A304F01230029006BBE060BA
:074D1F00037F01227F002247
:104C92009006BAEBF07B017A0679BA900618E4F036
:0A4CA200A304F0E4A3F01236EA22A6
:104A9F00C00790063CE0FFA3E0900604CFF0A3EF21
:104AAF00F0D0071230029006BBE060037F01227F37
:024ABF000022D3
:104CAC00C007900644E0FFA3E0900618CFF0A3EFF6
:0A4CBC00F0E4A3F0D0071236EA225C
:104B6900A2AFE433FCC2AF758F0175B7A575B7F174
:104B79008F828E83EDF0E4F58FAF04EF24FF92AFBF
:014B89002209
:104B8A00A2AFE433FDC2AF758F0375B7A575B7F150
:0F4B9A008F828E83E4F0F58FAF05EF24FF92AF8B
:014BA90022E9
:10442100900695EEF0A3EFF0A3ECF0A3EDF0EB4ACC
:104431006039900695E0FEA3E0FFA3E0FCA3E0F560
:10444100828C83E0FD124B69EB1B70011A90069878
:10445100E004F07006900697E004F0900696E00400
:0C446100F070CB900695E004F080C322C0
:084EE300E4900051F0A3F0225D
:1049A100900051E0FEA3E0FF124B8A900051E0FE1F
:1049B100A3E0FF7C007D537B007A02124421E49046
:0649C1000051F0A3F022FA
:0A3D8D00A905900669EEF0A3EFF01F
:103D9700EE54FEFE900051E0FCA3E0FD7002EE6CD5
:103DA7006057ED4C60031249A1900669E0FEEE549E
:103DB700FEFE7F00900051F0A3EFF090066BEEF04F
:103DC700A3EFF0A37400F0A37453F07E0290066B88
:103DD700E475F0011223A985F082F583E493FD9041
:103DE700066DE475F0011223A985F082F583EDF0E5
:103DF700EF1F70011EEF4E70D4900669E0FCA3E040
:103E0700FDEC5401FC74532DF58274003CF583E9F5
:013E1700F0BA
:013E18002287
:1044B400900655EEF0A3EFF0A3EBF0A3EAF0A3E926
:1044C400F090065A74FFF5F01223A945F060269087
:1044D4000655E475F0011223A9AFF0FE900657E0EB
:1044E400FBA3E475F0011223A9A9F0FA12226CFDD2
:0644F400123D8D80CC2278
:1033C4000212000048048C023602340237023548E7
:1033D4000484023202330130003048049402300283
:1033E40031013100314C04BC01320133013400326B
:1033F400003300344C04C80137013601350037006E
:033404003600355A
:104DB8007F008F178F147F1B8F188F157F368F19E1
:034DC8008F162221
:0645C5007B017D047C0077
:1045CB0090067BEBF0A3EAF0A3E9F0A3ECF0A3EDEC
:1045DB00F090067E74FFF5F01223A945F060189059
:1045EB00067BE0FBA3E475F0021223A9A9F0FAE421
:0845FB00FDFC123BD480DA2222
:10463D007E007F207D007B017A04799C122462121A
:10464D004DB87A04798C1245C57A0479841245C522
:10465D007B017A0479941245C77B017A0479BC7D7C
:09466D00067C001245CB0237F176
:0A3BCA007B0135F0FAE0FCA3E0FDFA
:103BD4009006B2ECF0A3EDF0C2AD12226C14602F8B
:103BE40014605424027075900001122285A814F206
:103BF4009006B2E0FEA3E0FFE804F8EEF208EFF26C
:103C0400E5142403F514641B7052751400804D9060
:103C14000001122285A815F29006B2E0FEA3E0FF8F
:103C2400E804F8EEF208EFF2E5152403F51564361E
:103C3400702A75151B8025900001122285A816F2A2
:103C44009006B2E0FEA3E0FFE804F8EEF208EFF21B
:103C5400E5162403F516B45103751636D2ADD21DFC
:013C6400223D
:0E3E9C0090065CEFF0A3ECF0A3EDF0A3EBF0CA
:103EAA00D394665018E0FD75F080A4FBED25E0FE82
:103EBA00E42BFFEE35F0900661F0A3EFF090065C7C
:103ECA00E075F002A4248CF9740435F0FA7B01A39E
:103EDA00123BCF90065FE0601390065CE075F0023B
:103EEA00A42484F97404900661123BCC900660E025
:103EFA00601E90065CE075F002A42494F9740435FF
:103F0A00F0FA7B01900660E07D0025E0FC123BD4CC
:013F1A002284
:053B29009006B4EFF06E
:103B2E00ED75F00AA42495F582E43402F583E0FEE7
:103B3E009006B5F0EF75F005A42458F582E4340331
:103B4E00F583E0FB3395E0FAEEFF7E00EB2FFFEE00
:103B5E003AFED3EF947FEE6480948040089006B5D1
:103B6E00747FF08014C3EE648094805007E4900656
:103B7E00B5F080059006B5EFF09006B4E0FF24088E
:103B8E00F876F0EF75F005A42456F582E43403F5CB
:103B9E0083E0FFED75F00AA42496F582E43402F575
:103BAE0083E0FD7C001238F8900660EFF09006B4CA
:0C3BBE00E0FFA3E0FB74FFFDFC023E9C56
:1019CC00EF25E025E0249CF582E43404F5837401D2
:1019DC00F00513E513AA127002051214FBEF25E0B3
:1019EC0025E0249EF582E43404F583EAF0A3EBF0C1
:1019FC00EF25E025E0249DF582E43404F583EDF039
:011A0C0022B7
:1049C700EF25E025E0249EF582E43404F583E0FA40
:1049D700A3E0FBC39511EA9510500A8A108B118F3B
:0649E7000DAF058F0F2249
:100AA700E49004D4F09004D4E0FFC394045029EFF9
:100AB70075F008A424D9F582E43404F583740FF0A3
:100AC700EF75F008A424DAF582E43404F583E4F042
:100AD7009004D4E004F080CDE49004D5F09004D5E0
:0A0AE700E0FFC39410400302162341
:100AF100EF75F00AA42493F582E43402F583E090C3
:080B010004FAF0700302161A59
:100B0900A37401F09004D5E075F00AA42494F58249
:100B1900E43402F583E09004FCF0E49004D4F0900E
:100B290004D4E0FFC3940840030215BEEF6003B488
:100B3900040DE4F50FF50EF50D74FFF510F511EF41
:100B490075F005A42440F582E43403F583E0FF90B1
:100B590004D5E0FEEF6E60030212379004D4E0FF83
:100B690075F005A42441F582E43403F583E07003AC
:100B7900020DA09004FAE064016035EF25E025E05C
:100B8900249CF582E43404F583E070030212379063
:100B990004D4E025E025E0249DF582E43404F583BE
:100BA900E0FE9004FCE0FDEE6D6003021237801C4C
:100BB900E50E60030212379004D4E0FF25E025E03A
:100BC900249CF582E43404F583E0600B9004FBE097
:100BD900FD1249C7021237750E019005B7E0FF9063
:100BE90004FBE0FEEF4E9005B7F09004D4E0FF90CF
:100BF90004FCE0FD1219CC9004D4E0FFC394044036
:100C090003020D90A3E075F00AA42495F582E4345B
:100C190002F583E0FD7C00EF75F005A42444F5821C
:100C2900E43403F583E0FF3395E0FEEF2DFFEC3E5E
:100C3900FE9004F7F0A3EFF0D3947FEE64809480E4
:100C4900400B9004F7E4F0A3747FF0800FC3900485
:100C5900F7E0648094805004E4F0A3F09004F7A3D3
:100C6900E0547FA3F0E49004D6F09004D6E0FFC3EB
:100C790094044003021237EF75F008A424DAF582D0
:100C8900E43404F583E06003020D239004D6E07593
:100C9900F008A424DAF582E43404F5837490F09022
:100CA90004F9E0FEEF75F008A424DCF582E43404CD
:100CB900F583EEF09004D4E075F005A42442F582A2
:100CC900E43403F583E0FF9004D5E075F00AA42429
:100CD90096F582E43402F583E0FD7C001238F89041
:100CE90004D6E0FE75F008A424DDF582E43404F5A9
:100CF90083EFF0EE75F008A424DAF582E43404F504
:100D090083C083C082E0FF9004D4E0FE7408A80683
:100D1900088002C313D8FC4F80599004D6E0FF75B0
:100D2900F008A424DAF582E43404F583E0FE54F0F3
:100D39006490704AEF75F008A424DCF582E4340469
:100D4900F583E0FF9004F9E0FDEFB505319004D695
:100D5900E075F008A424DAF582E43404F583C0834D
:100D6900C0829004D4E0FF7408A807088002C31366
:100D7900D8FC4ED082D083F09004D67404F090044D
:100D8900D6E004F0020C739004D4E024FCFFA3E045
:100D9900FD123B290212379004FAE0FC9005B7B422
:100DA900030CE0FE9004FBE0F4FDEE5D8009E0FF3A
:100DB9009004FBE0FEEF4E9005B7F09004D4E0FFFD
:100DC900C3940440030210E4EC64036003020F5C63
:100DD900A3E075F00AA42495F582E43402F583E0D2
:100DE900FD7C00EF75F005A42444F582E43403F595
:100DF90083E0FF3395E0FEEF2DFFEC3EFE9004F714
:100E0900F0A3EFF0D3947FEE64809480400B9004BC
:100E1900F7E4F0A3747FF0800FC39004F7E06480D7
:100E290094805004E4F0A3F09004F7A3E0547FA366
:100E3900F0E49004D6F09004D6E0FFC39404400394
:100E4900021237EF75F008A424DAF582E43404F5C8
:100E590083E06003020EEF9004D6E075F008A42445
:100E6900DAF582E43404F5837480F09004F9E0FE45
:100E7900EF75F008A424DCF582E43404F583EEF080
:100E89009004D4E075F005A42442F582E43403F516
:100E990083E0FF9004D5E075F00AA42496F582E476
:100EA9003402F583E0FD7C001238F89004D6E0FEA8
:100EB90075F008A424DDF582E43404F583EFF0EE3F
:100EC90075F008A424DAF582E43404F583C083C0FC
:100ED90082E0FF9004D4E0FE7408A806088002C3EB
:100EE90013D8FC4F80599004D6E0FF75F008A4246C
:100EF900DAF582E43404F583E0FE54F06480704A44
:100F0900EF75F008A424DCF582E43404F583E0FFEE
:100F19009004F9E0FDEFB505319004D6E075F008CD
:100F2900A424DAF582E43404F583C083C0829004F2
:100F3900D4E0FF7408A807088002C313D8FC4ED078
:100F490082D083F09004D67404F09004D6E004F0C3
:100F5900020E3F9004D5E075F00AA42495F582E4C9
:100F69003402F583E0FF7E009004D4E075F005A417
:100F79002444F582E43403F583E0FD3395E0FCED88
:100F89002FFFEE3CFE9004F7F0A3EFF0D3947FEE31
:100F990064809480400B9004F7E4F0A3747FF080A0
:100FA9000FC39004F7E0648094805004E4F0A3F048
:100FB9009004F7A3E0547FA3F0E49004D6F09004E2
:100FC900D6E0FFC394044003021237EF75F008A47A
:100FD90024DAF582E43404F583E0600302107790A3
:100FE90004D6E075F008A424DAF582E43404F58324
:100FF9007490F09004F9E0FEEF75F008A424DCF594
:1010090082E43404F583EEF09004D4E075F005A48D
:101019002442F582E43403F583E0FF9004D5E075BA
:10102900F00AA42496F582E43402F583E0FD7C00FD
:101039001238F89004D6E0FE75F008A424DDF58294
:10104900E43404F583EFF0EE75F008A424DAF582B0
:10105900E43404F583C083C082E0FF9004D4E0FE49
:101069007408A806088002C313D8FC4F805990045D
:10107900D6E0FF75F008A424DAF582E43404F58398
:10108900E0FE54F06490704AEF75F008A424DCF592
:1010990082E43404F583E0FF9004F9E0FDEFB5053F
:1010A900319004D6E075F008A424DAF582E434041A
:1010B900F583C083C0829004D4E0FF7408A80708B0
:1010C9008002C313D8FC4ED082D083F09004D6742A
:0B10D90004F09004D6E004F0020FC702
:1010E400E4900503F0A3F09004FAE0B4030AE4905A
:1010F40004FDF0A3F00211D674FF9004FDF0A3F0F8
:10110400900503E4F0A374F0F09004D4E075F005C6
:10111400A42442F582E43403F583E0FF9004D5E08F
:1011240075F00AA42496F582E43402F583E0FD7C8C
:10113400001238F8EF25E09004FFF0A3E4F09004E7
:10114400D4E075F005A42444F582E43403F583E087
:10115400FF3395E0FE9004D5E075F00AA42495F5DC
:1011640082E43402F583E02FFFE43EFE900506F0AE
:10117400A3EFF0D3947FEE64809480400B90050637
:10118400E4F0A3747FF0800FC3900506E0648094BC
:10119400805004E4F0A3F0900506E0FCA3E0FD54C5
:1011A4007F25E0900501F0A3E4F0D3ED9466EC64B0
:1011B400809480501D900506E0FEA3E07807C333B9
:1011C400CE33CED8F9FF900502E02FF0900501E070
:1011D4003EF09004D4E024FC900505F0900503A3B0
:1011E400E0FFA3E0FE2408F8A6079004FAE06402F6
:1011F4006010EE75F002A4248CF974049004FD12BE
:101204003BCA9004FAE064036029900505E075F098
:1012140002A42484F97404900501123BCA900505C4
:10122400E075F002A42494F9740435F0FA9004FFF4
:03123400123BCF9B
:101237009004FBE025E0F09004D4E0FF640360082D
:10124700EF640760030215B59004FAE064017003C8
:1012570002140DE50F700302140D9005B7E0FFE5CA
:101267000FF4FEEF5EF0E50D25E025E0249CF58206
:10127700E43404F583E4F0E50DC39404400302135A
:10128700FA9004D5E075F00AA42495F582E43402B7
:10129700F583E0FF7E00E50D75F005A42444F58293
:1012A700E43403F583E0FD3395E0FCED2FFFEE3CDE
:1012B700FE9004F7F0A3EFF0D3947FEE6480948060
:1012C700400B9004F7E4F0A3747FF0800FC3900401
:1012D700F7E0648094805004E4F0A3F09004F7A34F
:1012E700E0547FA3F0E49004D6F09004D6E0FFC367
:1012F700940440030215B5EF75F008A424DAF582CB
:10130700E43404F583E060030213989004D6E07593
:10131700F008A424DAF582E43404F5837480F090AD
:1013270004F9E0FEEF75F008A424DCF582E4340448
:10133700F583EEF0E50D75F005A42442F582E4345B
:1013470003F583E0FF9004D5E075F00AA42496F531
:1013570082E43402F583E0FD7C001238F89004D66D
:10136700E0FE75F008A424DDF582E43404F583EF8C
:10137700F0EE75F008A424DAF582E43404F583E08E
:10138700FFAE0D7408A806088002C313D8FC4F806F
:10139700529004D6E0FF75F008A424DAF582E4340D
:1013A70004F583E0FE54F06480703FEF75F008A405
:1013B70024DCF582E43404F583E0FF9004F9E0FDD2
:1013C700EFB505269004D6E075F008A424DAF58277
:1013D700E43404F583AF0D7408A807088002C3132B
:1013E700D8FC4EF09004D67404F09004D6E004F0D4
:1013F7000212F1E50D24FCFFE4900660F0FBFDFC12
:10140700123E9C0215B5E50E60030215B5E50F7097
:10141700030215B59005B7E0450FF09004FCE0FD19
:10142700AF0D1219CCE50DC3940440030215A89023
:1014370004D5E075F00AA42495F582E43402F58317
:10144700E0FF7E00E50D75F005A42444F582E43441
:1014570003F583E0FD3395E0FCED2FFFEE3CFE90B6
:1014670004F7F0A3EFF0D3947FEE64809480400BF1
:101477009004F7E4F0A3747FF0800FC39004F7E0C3
:10148700648094805004E4F0A3F09004F7A3E05440
:101497007FA3F0E49004D6F09004D6E0FFC3940451
:1014A70040030215B5EF75F008A424DAF582E43499
:1014B70004F583E060030215469004D6E075F00852
:1014C700A424DAF582E43404F5837490F09004F9E7
:1014D700E0FEEF75F008A424DCF582E43404F5831C
:1014E700EEF0E50D75F005A42442F582E43403F52A
:1014F70083E0FF9004D5E075F00AA42496F582E412
:101507003402F583E0FD7C001238F89004D6E0FE43
:1015170075F008A424DDF582E43404F583EFF0EEDA
:1015270075F008A424DAF582E43404F583E0FFAE0D
:101537000D7408A806088002C313D8FC4F80529088
:1015470004D6E0FF75F008A424DAF582E43404F544
:1015570083E0FE54F06490703FEF75F008A424DC3C
:10156700F582E43404F583E0FF9004F9E0FDEFB57C
:1015770005269004D6E075F008A424DAF582E43451
:1015870004F583AF0D7408A807088002C313D8FCBD
:101597004EF09004D67404F09004D6E004F00214E0
:1015A7009FE50D24FCFF9004D5E0FD123B29900434
:1015B700D4E004F0020B28E49004D6F09004D6E0BF
:1015C700FF75F008A424DAF582E43404F583E060BB
:1015D7002FEF75F008A424D7F9740435F0FA7B01CE
:1015E7007D08124E869004D6E075F008A424DAF53B
:1015F70082E43404F583E4F09004D6E004F080BC80
:101607009004D5E075F00AA42493F582E43402F53A
:0316170083E4F079
:0C161A009004D5E004F0020AE4024585CB
:1037F100201D030238F7C21DE514B5170EE515B5F6
:0B3801001809E516651970030238F77E
:10380C00C283E516B519089006A474F0F08020A8C0
:10381C0019E29006A4F0E804F8E2FF08E2A3CFF066
:10382C00A3EFF0E5192403F519B45103751936E427
:10383C00FF124EEB9006A4E0FF124EEB9006A5E0B3
:10384C00FF124EEB9006A5A3E0FF124EEBE515B56B
:10385C0018089006A474F0F08020A818E29006A432
:10386C00F0E804F8E2FF08E2A3CFF0A3EFF0E518CC
:10387C002403F518B4360375181BE4FF124EEB90B5
:10388C0006A4E0FF124EEB9006A5E0FF124EEB9063
:10389C0006A5A3E0FF124EEBE514B517089006A49D
:1038AC0074F0F08020A817E29006A4F0E804F8E287
:1038BC00FF08E2A3CFF0A3EFF0E5172403F517B44C
:1038CC001B03751700E4FF124EEB9006A4E0FF12E9
:1038DC004EEB9006A5E0FF124EEB9006A5A3E0FF81
:0838EC00124EEB124F15D283BE
:0438F4000237F9227C
:104AC10074082FF8E6601A16E67016EF75F002A466
:104AD100248CF9740435F0FA7B017D007C80123B53
:024AE100D422DD
:031A12000242D6B7
:1042D600C0E0C0F0C083C082C0D075D000C000C0AE
:0D42E60001C002C003C004C005C006C0072F
:1042F300C2CF9006BCE4F09006BCE0FFC394045028
:0C4303000B124AC19006BCE004F080EBF5
:10430F00D007D006D005D004D003D002D001D00002
:0B431F00D0D0D082D083D0F0D0E032AC
:104E100000FF0100010000FFFF0000010001FF0092
:073407004205B50000C118E9
:053E1900900699EFF096
:103E1E00E54C2401FFE4354BFAA907A37401F0A386
:103E2E00EAF0A3E9F090069AE0FBA3E0FAA3E0F92A
:103E3E0074019005CC6B7008E965827003EA6583A6
:103E4E00700D90069A04F0A37405F0A374B8F09068
:103E5E00069AE0FBA3E0FAA3E0F9E54D854E8385D3
:103E6E004F826B7008E965827003EA6583601E906D
:103E7E000699E0854C82854B83F090069AA3E0FA72
:0D3E8E00A3E0AE028E4BF54C900699E0F0DB
:013E9B002204
:074D52009006A7E0FFAD4948
:0E4D5900EB5F6009ED5B6005AF03123E1922AF
:0D4E480075BC4475E8C075BA1F75D108220D
:1043D00053E6EFE54D854E83854F826401700AE513
:1043E0004C65827004E54B65837003FF802FAB4DF5
:1043F000054FE54FAA4E7002054E14F912226CFFCC
:1044000074019005CC6B700AE54F65827004E54E2F
:1044100065837009754D01754E05754FB843E610FB
:014420002279
:1048AC0053E6EFE54D854E83854F826401700AE532
:1048BC004C65827004E54B65837003FF800AAB4D39
:0B48CC00AA4EA94F12226CFF43E61019
:0148D70022BE
:104A5900EFD394B840047E108016EFD394784004C5
:104A69007E04800CEFD3945040047E018002E4FE62
:024A7900AF0686
:014A7B002218
:031A240002314D3F
:10314D00C0E0C0F0C083C082C0D075D000C001C047
:0F315D0002C003C005C006C00720DF0302321204
:10316C009006A8E5BEF0D2ECA217B3921730170D5B
:10317C0075BB04E0FF124A598F4902321075BB032C
:10318C009006A8E0FF124A59EF25E04249E549654F
:10319C00536012E54965539006A7F0543F600375E0
:1031AC005103854953E551605B1551E5517055E567
:1031BC005265499006A7F09005B5E07002A3E06057
:1031CC0006E5497002D2187B01124D527B02124D5A
:1031DC00529006A7E0FF7B04AD49124D599006A70B
:1031EC00E0FF7B08AD49124D599006A7E0FF7B101C
:1031FC00AD49124D599006A7E0FF7B20AD49124D09
:06320C0059854952C2DFA2
:0632120020D80330D9585A
:103218009006A7E590F0C2D9C2D8E0FD65505403E6
:103228006046E55075F004A47E00540CFFED54038D
:10323800FDEF4D2410F582EE344EF583E493FF90B4
:1032480006A8F0A3E54AF0EF254AF54AE0654A30BA
:10325800E1109006A8E0B401047F0980027F0A12F9
:083268003E199006A7E0F550A5
:10327000D007D006D005D003D002D001D0D0D08264
:07328000D083D0F0D0E03252
:0C4E620075DA3175DB3175D989D2DE229A
:104C2600124E627B017A0579B88B4D8A4E894F8A7E
:0B4C36004B894CE49005B7F002458567
:064F1500E5A120E7FB22EC
:084EEB00E5A120E7FB8FA322E3
:104585007D017C00E4FB90054EE0FFEBC39F500AE4
:10459500ED25E0FDEC33FC0B80EC301504EC4440DC
:1045A500FCC2AFD2839005B7E0F4FF124EEBECF4FA
:0F45B500FF124EEBEDF4FF124EEB124F15D2AF8B
:0145C40022D4
:10340E006054042F00010204081000000304180089
:10341E00000000001F000000000018040300000060
:10342E000010080402010000040A0A111100000134
:10343E000102021C00001C02020101000010100813
:10344E0008070000070808101000001818001818C8
:08345E00000018180318180003
:064F1B001247898FA0225D
:0D4E20007FC87E00EF1F70011EEF4E70F77F
:014E2D002262
:104DEE007F38124D7C7F06124D7C7D0EE4FF024E05
:014DFE006E46
:104D7C009006BDEFF0124D67EF20E7F99006BDE00D
:044D8C00FF024D9045
:104D670075A0FFC296D295D2977F14DFFEAFA0122F
:044D77004789C2970F
:014D7B002215
:054F33007F01024D7C2E
:104D9000124F1B124E20C296C295D297124E20C2BD
:044DA00097024E2008
:104DFF00124F1BC295D297D296124E20C297024ED7
:014E0F002082
:0C4E6E00900483E05FF04DFFF0024D7CEB
:0F4A7C00A3E475F0011223A9A9F0FA12226CFF2E
:104A8B009006BEEFF0124D67EF20E7F99006BEE0FF
:044A9B00FF024DFFCA
:104A12009006AAEBF0A3EAF0A3E9F09006AAE0FB65
:104A2200A3E0FAA3E0F912226C60089006AA124AE7
:044A32007C80E8227A
:1046E80090066FEBF0A3EAF0A3E9F0124F33E4FD74
:1046F800FF124E7A90066FE0FBA3E0FAA3E0F912EE
:104708004A12E4FD7F01124E7A900672E0FBA3E0A4
:07471800FAA3E0F9024A12C6
:0C4E7A00EF75F040A42D2480FF024D7C59
:08428000900675EFF0A3EDF0CC
:10428800E075F008A42440FF124D7C900675E054B8
:104298007F75F007A4242FF9740435F0FA90067896
:1042A8007401F0A3EAF0A3E9F0900676E0900675B1
:1042B800F09006777407F0900677E0FF14F0EF604F
:0E42C80008A3E0FB124A7C80EEE4FF024A8B62
:10478900E4F55DF55EF55CAE5C7480A80608800210
:10479900C313D8FCF55D5F600FAE5C7401A8060811
:1047A9008002C333D8FC425E055CE55CB408D8AF2F
:0147B9005EA1
:0147BA0022DC
:10346600C10EC10F4E02550002000200020002000A
:10347600010001000241033F004A02896030201822
:0E348600100C080604034102530041025400DA
:031A1500D20F22CB
:034F3800C20F2283
:104BE9007E007FA07D007B017A027993122462E422
:0F4BF9009005B7F0C20DC20AF55FF560C20E223B
:091A1B00124BE912463DD20922EA
:0C4E8600300F08E4900667F0124540224F
:1038F800EF14B4090040030239BF90391075F00382
:10390800A4C58325F0C5837302396402392E0239B0
:103918005B02392B02396F02394902393302398087
:1039280002399E0239BA7D500239BF74C12DFD7427
:10393800FF3CC3648094805002E4FDED25E0FD80E7
:103948007174C12DFD74FF3CC3648094805041E4C0
:10395800FD803DC374809DFDE49C8001ECA2E713CB
:10396800ED13243CFD8050D3ED943FEC64809480AB
:103978004004747F9DFD8018C374809DFDE49CFC09
:1039880074C12DFD74FF3CC3648094805002E4FD33
:10399800ED25E0FD8021C374809DFDE49CFC74C18D
:1039A8002DFD74FF3CC3648094805002E4FDED2536
:0A39B800E0FDC374809DFDAF052201
:104C4100E49006BFF09006BFE0FFC39404500B123E
:0A4C510044FA9006BFE004F080EB87
:014C5B002236
:0244FA00AD070C
:1044FC00900648740FF07408A807088002C313D8FC
:10450C00FC44B0900649F090064B741FF0ED75F02A
:10451C0005A42443F582E43403F583E090064CF0C3
:10452C00300F107B017A067946E4900667F07D081F
:03453C00124540E5
:01453F002259
:0C401200F583E0FEC4540FFFEE540FFDD8
:10401E00AB05AA0774892BF582E43402F583E0FD23
:10402E003395E0FCE56024FFFFE55F34FFFE1223CD
:05403E005DED4C704631
:1040430074892BF582E43402F583E0FD3395E0FCBB
:10405300E56024FFFFE55F34FFFE1223089006B6F8
:10406300EEF0A3EFF0E004F070069006B6E004F083
:104073000AEAFD7C009006B6E0FEA3E0FF122308E7
:06408300ED4C7002D32297
:02408900C32250
:102D5D00E49006C0F09006C0E0FFC3940640030265
:102D6D002EB2EF75F005A42468F582E43403F583E3
:102D7D00E064106003022EA99006C0E075F005A472
:102D8D002469F582E4340312401250319006C0E0FC
:102D9D0075F002A424BCF9740435F0FA7B0174FFBC
:102DAD00FDFC123BD4900253E0FF9006C0E0FE7490
:102DBD0001A806088002C333D8FC4F80499006C095
:102DCD00E0FD74017E00A805088005C333CE33CE27
:102DDD00D8F9FF900253E0FBEF5B602EED75F0022A
:102DED00A424BCF9740435F0FA7B01E4FDFC123B1C
:102DFD00D4900253E0FF9006C0E0FEE4A8060880E0
:102E0D0002C333D8FC5F900253F09006C0E075F01A
:102E1D0005A4246AF582E434031240125031900661
:102E2D00C0E075F002A424C8F9740435F0FA7B01F2
:102E3D0074FFFDFC123BD4900254E0FF9006C0E0FD
:102E4D00FE7401A806088002C333D8FC4F80499058
:102E5D0006C0E0FD74017E00A805088005C333CED1
:102E6D0033CED8F9FF900254E0FBEF5B602EED7589
:102E7D00F002A424C8F9740435F0FA7B01E4FDFCDA
:102E8D00123BD4900254E0FF9006C0E0FEE4A80689
:102E9D00088002C333D8FC5F900254F09006C0E066
:052EAD0004F0022D629B
:012EB20022FD
:0E27A3009005CCEFF0A3ECF0A3EDF0A3EBF06B
:1027B1009005D174B0F0A374E0F09005D5740FF0DA
:1027C100E49005D0F09005D0E0FFC39404505DEF94
:1027D10075F005A42440F582E43403F583E0FF900D
:1027E10005CFE0FEEF6E703C9005CCE0701C9005CB
:1027F100D2E0FF9005D0E0FE7408A806088002C36D
:1028010013D8FC4F9005D2F0801A9005D1E0FF90CB
:1028110005D0E0FE7408A806088002C313D8FC5F47
:102821009005D1F09005D0E004F08099E49005D0B6
:10283100F09005D0E0FFC3940640030228E9EF754C
:10284100F005A42469F582E43403F583E0FF9005E3
:10285100CCE0FEEF6E70379005D0E0FF75F005A477
:102861002468F582E43403F583E0FE9005CFE0FDB2
:10287100EEB5051AEF75F002A424BCF9740435F025
:10288100FA7B019005CDE0FCA3E0FD123BD490055D
:10289100D0E0FF75F005A4246AF582E43403F583E2
:1028A100E0FE9005CCE0FDEE6D7034EF75F005A40F
:1028B1002468F582E43403F583E0FF9005CFE0FE60
:1028C100EFB5061BA3E075F002A424C8F974043522
:1028D100F0FA7B019005CDE0FCA3E0FD123BD49022
:1028E10005D0E004F00228329005D1E0FF540F60DA
:1028F100299005D6EFF09005CCE09005D8F0900531
:10290100CDA3E09005D9F0300F107B017A0579D382
:10291100E4900667F07D081245409005D2E0FF542F
:102921000F60389005D6EFF09005CDE0FCA3E0FDF7
:10293100AE047802CEC313CE13D8F9547F9005D8D4
:10294100F0ECC313547FA3F0300F107B017A0579AB
:10295100D3E4900667F07D081245409005CCE06411
:10296100426003022A4F9005CFE090033FF0A20A94
:10297100920DC39005CDE094804003022A4DC20A16
:06298100200D03022A4FA5
:062987009005DB7403F073
:10298D009005DC7403F09005DCE0FFC36480948057
:10299D004058EF3395E0FEEF25E0FFEE33FE900358
:1029AD003FE0FD75F00AA42496F582E43402F58328
:1029BD00E5822FF582E5833EF583E4F074372FF53C
:1029CD008274033EF583E0FCED75F00AA42495F5C1
:1029DD0082E43402F583E5822FF582E5833EF583AB
:1029ED00ECF09005DCE014F0809C90033FE0FD7569
:1029FD00F00AA42493F582E43402F5837403F09075
:102A0D0005DBE0FF3395E0FEEF25E0FFEE33FE74CE
:102A1D00372FF58274033EF583E0FFED75F00AA4C0
:0E2A2D002494F582E43402F583EFF0120AA738
:102A3B009005DBE014F0E0C364809480400302292E
:022A4B008D22DA
:022A4D00D20AAB
:012A4F002264
:1024AE00C21E90061D740FF0EF122436258980246B
:1024BE00DC9026EDA026FFB02717C026CCE02766BD
:1024CE00F82736FA275AFB274EFC0000278C90027D
:0724DE006DE0700302258987
:1024E5009006237402F0900264E075F00AA4FDAC36
:1024F500F02495F974023CFA7B01900623E0FF3342
:1025050095E0FEEF25E0FFEE33FEE92FF9EA3EFA0E
:10251500C002C00174972DF974023CFAE92FF9EA5B
:102525003EA801FC7D01D001D0027E007F0212226F
:1025350046900623E014F0E0C36480948050A79091
:10254500026CE0FF900264E0FE75F00AA42495F5A4
:1025550082E43402F583EFF090026DE0FDEE75F054
:102565000AA42496F582E43402F583EDF0EE75F0C5
:102575000AA42493F582E43402F5837401F0D209A8
:04258500EE0226BA82
:10258900300A629006237402F0900623E0FFC364C8
:102599008094804044EF3395E0FEEF25E0FFEE3371
:1025A900FE74372FF58274033EF583E0FD74392FED
:1025B900F58274033EF583EDF074382FF5827403C8
:1025C9003EF583E0FD743A2FF58274033EF583ED01
:1025D900F0900623E014F080B090026CE09003378D
:1025E900F0E4A3F022E4900623F0900623E0FFC371
:1025F9006480948440030226B1EF3395E0FEEF2511
:10260900E0FFEE33FE900264E075F00AA42495F52C
:1026190082E43402F583E5822FF582E5833EF58372
:10262900E0FF90026CE0FEEF6E7074900623E0C349
:10263900648094835053900264E075F00AA4FDAC61
:10264900F02497F974023CFA7B01900623E0FF33EA
:1026590095E0FEEF25E0FFEE33FEE92FF9EA3EFAB9
:10266900C002C00174952DF974023CFAE92FF9EA08
:102679003EA801FC7D01D001D0027E007F0212221A
:1026890046900623E004F080A2900264E075F00A07
:10269900A42493F582E43402F5837403F0D20990FB
:1026A9000623E004F00225F390026CE0FF90026437
:1026B900E075F00AA42494F582E43402F583EFF07E
:0326C90002278C59
:1026CC0090026CE075F004A4FDA3E025E0FEE42D7F
:1026DC00FFEE35F0FEAD07FC900264E0FBE4FF80FA
:1026EC002590026DE07D0025E0FC900264E0FB7F0C
:1026FC0001801390026CE02402FFA3E07D0025E032
:10270C00FC900264E0FB1227A3807590026CE0FF42
:10271C00C3941E506B90061E74C0F0900264E0903F
:10272C00061FF0A3EFF0D21E8056D20EE490025397
:10273C00F0A3F090061E74FAF0D21EE4F55FF5607B
:10274C00803E90061E74FCF0D21EC20E80329006A3
:10275C001E74FBF0D21ED20E8026300E2390061E65
:10276C0074F8F0D21E0560E560AE5F7002055F1470
:10277C00B4000AEEB40306755F00756001122D5D9E
:10278C00301E13300F107B017A06791BE49006671C
:06279C00F07D081245402B
:0127A2002214
:1040FA00AE07EF7008900265F0A3F08057EE54F017
:10410A00900263F0EE540FA3F0EEC394F0402690B1
:10411A000263EEF0B4F00BE4900269F0900267F0EB
:10412A00A3F0EEC394F85005E490026AF09002649A
:10413A0074FFF0801F90026AEEF0C4540F25E02449
:10414A0045F582E43402F583E0FFA3E0900265CFEF
:0C415A00F0A3EFF0E4900267F0A3F02265
:103F1B009006C1EFF030E72AE0FFB4FF0122EF6417
:103F2B00F8600EEF64FA6009EF64FC6004EFB4FB19
:103F3B00030224AE9006C1E0C394F750509006C123
:103F4B008046900265E07002A3E060419006C1E0FC
:103F5B00FF900269E02FF0900267E475F0011223E5
:103F6B00A9FC746C25F0F58274023CF583EFF0909C
:103F7B00026574FFF5F012239345F0701090026305
:0E3F8B00E0FF1224AE90026AE0FF1240FA221C
:043494004103CC0024
:1034C800E49006ADF0A37403F0E4A3F0124EE37E9B
:1034D800E07F017B017A0679AE90065AE4F0A304F6
:1034E800F01244B47E007F467D007B017A03794068
:1034F800122462E49006ADF09006ADE0FFC3940E8E
:10350800400302358EEFC39408EF75F0055050A4C0
:103518002440F582E43403F58374FFF0EF75F00579
:10352800A42443F582E43403F5837432F0EF75F094
:1035380005A42442F582E43403F583E4F0EF75F042
:1035480005A42441F582E43403F583E4F0EF75F033
:1035580005A42444F582E43403F583E4F0800DA443
:103568002440F582E43403F58374FFF0EF75F00529
:10357800A42443F582E43403F5837432F09006AD55
:10358800E004F0023500E49006ADF09006ADE0FFEF
:10359800C3941E502A75F046EFA42402F582E5F084
:1035A80034E0AF82FE7B017A03794090065AE4F05A
:1035B800A37446F01244B49006ADE004F080CC7ECB
:1035C800E07F007B017A0679AF90065AE4F0A30405
:0735D800F01244B40249A106
:064F2100E49003CCF02235
:074F02009003CC7401F022C2
:104DA40020191030150D9003CCE07007AF1F124B83
:044DB40027D21922C7
:104CF70090E000E493F46007A3E493640360031275
:084D070034C8E4F561C2192271
:10492C00E561C3941E501FE56175F046A42402F99D
:10493C0074E035F0FA7BFF78407C037D017E007FCC
:07494C0046122246C21922A7
:10481F00E561C3941E5029124EE375F046E561A47D
:10482F002402F582E5F034E0AF82FE7B017A037952
:10483F004090065AE4F0A37446F01244B41249A112
:01484F002246
:0B4EA800121A1B12481FC219024BE92E
:0539C2009005DEEDF0B0
:1039C7009005E0E004F09005E3EFF0A3EBF090053D
:1039D700DEE0FF9005E3E0FED39F4003023A7575F2
:1039E700F046EEA42402F582E5F034E0AF829005BC
:1039F700E5F0A3EFF09005E4E075F046A42402F5A6
:103A070082E5F034E0AF829005E7F0A3EFF0E490B1
:103A170005E1F0A3F09005E7E475F0011223A9AFE3
:103A2700F0FE9005E5E0FCA3E0F5828C83E493FDCE
:103A3700123D8D9005E6E004F070069005E5E00480
:103A4700F09005E2E004F070069005E1E004F0C3B1
:103A57009005E2E094469005E1E0940040B71249F2
:0E3A6700A19005E3E004F0A3E004F00239D5DD
:013A7500222E
:052BEB00900624EDF04E
:102BF000900629EFF0A3EBF0900624E0FF90062961
:102C0000E0D39F4003022D5CA3E075F046A42402AC
:102C1000F582E5F034E0AF82900625F0A3EFF0E412
:102C200090062BF0A3F090062BE0FEA3E0FFC394E8
:102C300046EE94005038900625E0FCA3E0F5828C27
:102C400083E493FD74862FF582E43403F583EDF07D
:102C5000900626E004F07006900625E004F0900649
:102C60002CE004F070C090062BE004F080B89006D1
:102C700029E075F046A42402F582E5F034E0AF8245
:102C8000900627F0A3EFF090062AE075F046A42402
:102C900002F582E5F034E0AF82900625F0A3EFF074
:102CA000E490062BF0A3F0900625E475F0011223C2
:102CB000A9AFF0FE900627E0FCA3E0F5828C83E448
:102CC00093FD123D8D900628E004F07006900627D3
:102CD000E004F090062CE004F0700690062BE0046F
:102CE000F0C390062CE0944690062BE0940040B789
:102CF000900629E075F046A42402F582E5F034E060
:102D0000AF82900627F0A3EFF0E490062BF0A3F03B
:102D100090062BE0FCA3E0FDC39446EC9400502CFD
:102D2000900627E475F0011223A9AFF0FE74862DFA
:102D3000F582E43403F583E0FD123D8D90062CE02E
:102D400004F070CC90062BE004F080C41249A190EE
:0C2D50000629E004F0A3E004F0022BF8D8
:012D5C002254
:0B3A7600900608EFF0A3EDF0A3EBF0CA
:103A8100A2AFE433A3F0C2AF124EFB900609E0FEF1
:103A9100900608E0FDEDFF900610EEF0A3EFF0E4D4
:103AA10090060CF090060AE0FF900610E0FCA3E0FF
:103AB100FD7B017A03798690063CE4F0A37446F01D
:103AC100124A9F900611E02446F0900610E034005F
:103AD100F090060CE075F046A42402F974E035F08C
:103AE100FAA374FFF0A3EAF0A3E9F0124EE3900603
:103AF1000DA3E0FAA3E0AE02FF7B017A0379869081
:103B0100065AE4F0A37446F01244B41249A1900697
:103B11000CE004F0E0C3941E408AAF1F124E3B90AC
:073B2100060BE024FF92AF48
:013B2800227A
:0B3CFA0090062DEFF0A3EDF0A3EBF01F
:103D0500A2AFE433A3F0C2AF124EFB90062EE0FE45
:103D150090062DE0FDEDFF900632EEF0A3EFF0E406
:103D2500900631F0900631E0FFC3941E504C75F0BB
:103D350046EFA42402F582E5F034E0AF82FE90065A
:103D450034F0FAA3EFF0FB90062FE0FF900632E087
:103D5500FCA3E0FDA9037BFF900644E4F0A37446B1
:103D6500F0124CAC900633E02446F0900632E03475
:103D750000F0900631E004F080AAAF1F124E3B9090
:073D85000630E024FF92AFBD
:013D8C002214
:0D4E55007E057F7A8E5A8F5B8E588F592212
:084EF300759810D2ACC2BC227C
:064F2700124E55024EF38C
:011A0D0022B6
:104DCB00E559655B7004E558655A60037F01227FE6
:024DDB000022B4
:104AE300055BE55BAE5A7002055A14F5828E83E0CE
:104AF300FF7498B55B0B7405B55A06755A05755B5B
:014B03007A37
:014B0400228E
:031A0F0002446D21
:10446D00C0E0C083C082C0D030982EC298855982DA
:10447D00855883E599F00559E55970020558B498AA
:10448D000BE558B4050675580575597AE559B55BB0
:10449D0008E558B55A03121A0D309902C299D0D0B9
:0744AD00D082D083D0E03281
:10328700205072696D6F2056657273696F6E2020CA
:10329700200020496E697469616C697A696E6720DC
:1032A700202020004D6F6E6F00506F6C790020500A
:1032B700570041667400253364006275733A2563CD
:1032C7002043683A2532642025730054722563250C
:1032D70032642046743A416E20566C3A2563005496
:1032E70072256325326420257325326420566C3A93
:1032F70025630046740046743A0058706F73653A48
:10330700252B3364202056656C3A2563004275737C
:103317003A2563204368616E3A436C6F636B0044E0
:1033270069763A2025642F252D3264203A202564BA
:103337002F252D3264004275733A25632043686157
:103347006E6E656C3A25326400436E74726C6C72F3
:10335700733A00000AFF432A000CFF471F0104FFCE
:103367004225010AFF4850010FFF4904000AFF43A5
:103377002A000CFF471F0108FF4225010FFF4904E0
:10338700000FFF437D010BFF4C5C010FFF4C7700E3
:103397000FFF437D0105FF47BB0107FF4676010C81
:0833A700FF47ED010EFF46AFE8
:10349800C1150F3441424344454647484A4B4C4DB9
:1034A8004E50000643FF32ABFF32B00624FF32B560
:0F34B800FF32B90A2A0102030406080C1018207B
:1048D800E4900552F0900551F0900550F090054F86
:1048E800F090054EF090067274FFF0A37432F0A3B6
:0C48F8007499F07BFF7A3279870246E861
:064F2D00E4900530F022C3
:103C65009006B8EEF0A3EFF0AF051DEF7003023C30
:103C7500F99006B8E0FEA3E0F5828E83A3A3E49352
:103C8500FB740193FA740293F9900530E0FF75F027
:103C950005A42436F582E43405F583EBF0A3EAF0B8
:103CA500A3E9F09006B8E0FAA3E0FBF5828A83E485
:103CB50093FEEF75F005A42434F582E43405F5830D
:103CC500EEF08B828A83740193FF900530E075F0E6
:103CD50005A42435F582E43405F583EFF09005302D
:103CE500E004F09006B9E02405F09006B8E0340051
:053CF500F0023C6D220D
:1041C600900553E0FBA3E0FAA3E0F912226CFE751A
:1041D600F005A42434F582E43405F583E0FFEE759A
:1041E600F005A42435F582E43405F583E0FD124E8E
:1041F6007A900553E0FBA3E0FAA3E0F912226C756E
:10420600F005A42436F582E43405F583E0F9A3E04D
:0F421600FAA3E0900531C9F0A3EAF0A3E9F02282
:10495300900553E0FBA3E0FAA3E0F912226C700781
:10496300900530E01222D4900553E0FBA3E0FAA3B4
:07497300E0F974FF0222B21B
:104BAA00900553E0FBA3E0FAA3E0F974011222B2E4
:104BBA0012226CFF900530E0B50704E41222D422D9
:0D46030035F0FA7B01E0FD7482900684F032
:10461000ED1222B212226CFF3395E0FE900684E088
:10462000FDD3EF9D7480F86E984003E0800B12225A
:0D4630006CC3648094805004E41222D422F4
:0B4B0500F583E0C4540FFFAD067B07F2
:104B10009006C2EFF0AF037B017A0679C2EF12462E
:074B20000C9006C2E0FF2229
:10432A0090054EE0FE75F005A42440F582E43403BE
:10433A00F583E02FF0EE75F005A42440F582E4340D
:10434A0003F583E0FFB4FE13EE75F005A42440F5EF
:10435A0082E43403F583740FF08015EFB41011EE84
:10436A0075F005A42440F582E43403F58374FFF064
:03437A00024DA44D
:10437D0090054EE0FE75F005A42440F582E434036B
:10438D00F583E02FF0EE75F005A42440F582E434BA
:10439D0003F583E0FFB4FE13EE75F005A42440F59C
:1043AD0082E43403F5837410F08015EFB41111EE2F
:1043BD0075F005A42440F582E43403F58374FFF011
:0343CD00024DA4FA
:10471F009006C3EFF090054EE075F005A42441F923
:10472F00740335F0FA7B019006C3E0FD90054EE06F
:10473F00C3940450047F0280027F01900684EFF03F
:06474F00124610024DA409
:1042250090054EE0FE75F005A42444F582E43403C0
:10423500F583E02FF0EE75F005A42444F582E4340F
:1042450003F583E0FFD3648094B04013EE75F00569
:10425500A42444F582E43403F5837430F08019C353
:10426500EF648094505011EE75F005A42444F58256
:0B427500E43403F58374D0F0024DA484
:104850009006C4EFF090054EE075F005A42443F9EE
:10486000740335F0FA7B019006C4E0FD9006847471
:1048700063F0124610124DA490054EE0FF0244FA78
:104904009006C5EFF090054EE075F005A42442F939
:10491400740335F0FA7B019006C5E0FD90068474BB
:0849240009F0124610024DA437
:1047BB00AE0790054EE075F005A42441F582E43474
:1047CB0003124B05EF540FC454F0FF90054EE075E8
:1047DB00F005A42441F582E43403F583E0540F4F34
:0247EB00F022BA
:10467600AE0790054EE075F005A42441F582E434BA
:1046860003F583E0540FFFAD067B09124B10EF5480
:104696000FFF90054EE075F005A42441F582E43441
:0946A60003F583E054F04FF0220B
:1047ED00AE0790054EE075F005A42442F582E43441
:1047FD0003124B05EF540FC454F0FF90054EE075B6
:10480D00F005A42442F582E43403F583E0540F4F00
:02481D00F02287
:1046AF00AE0790054EE075F005A42442F582E43480
:1046BF0003F583E0540FFFAD067B09124B10EF5447
:1046CF000FFF90054EE075F005A42442F582E43407
:0946DF0003F583E054F04FF022D2
:104C5C009006C6EFF090054EE075F005A42441F9DE
:0B4C6C0074039006C6124603024DA41C
:104C77009006C7EFF090054EE075F005A42442F9C1
:0B4C870074039006C7124603024DA400
:10408B0090069DEBF0A3EAF0A3E9F0A3EDF0C39447
:10409B0002502EE075F003A42424F8860308E6FAF8
:1040AB0008E6F9C003C00290069DE0FBA3E0FAA36B
:1040BB00E0F8AC02AD03D002D0037E007F030222F6
:1040CB004690050B74FFF0A37432F0A374BDF0900F
:1040DB0006A0E024FEFEE434FF90050EF0A3CEF024
:0F40EB0090069DE0FBA3E0FAA3E0F9121E7622F7
:101A2700124F2D90054EE0FFC394084003021C7B24
:101A3700EF75F005A42442F582E43403F583E0FF53
:101A47007D0112428090050B74FFF0A37432F0A35E
:101A570074C1F090054EE0FF2434F8E690050EF0CF
:101A6700EF75F005A42440F582E43403F583E02400
:101A770001FF90050FE4F0A3EFF090054EE075F03D
:101A870005A42441F582E43403F583E075F003A44B
:101A97002443F8860308E6FA08E6F9900511EBF007
:101AA700A3EAF0A3E9F07B017A057956121E769036
:101AB700054EE0FFC394044003021C2AEF75F005AE
:101AC700A42444F582E43403F583E07D0230E7047F
:091AD7007F0B80027F0A1242809D
:101AE00090054EE0FF75F005A42443F582E434032D
:101AF000F583E0FD7C00900578ECF0A3EDF0643216
:101B0000705190050B74FFF0A37432F0A374D2F0FF
:101B1000A37402F0EF75F005A42444F582E43403C5
:101B2000F583E0FF5480FD3395E04D6006EFF4044B
:101B3000FF801390054EE075F005A42444F582E47F
:101B40003403F583E0FFEF3395E090050FF0A3EF4A
:101B5000021C03900578E0FEA3E0FFD39432EE640C
:101B60008094804005E024CE8011C3EF9432EE646F
:101B7000809480500E900579E024CFF0900578E0B5
:101B800034FFF090050B74FFF0A37432F0A374E6F9
:101B9000F0A37402F090054EE075F005A42444F51E
:101BA00082E43403F583E0FF5480FD3395E04D601B
:101BB00006EFF404FF801390054EE075F005A424B1
:101BC00044F582E43403F583E0FFEF3395E09005BC
:101BD0000FF0A3EFF0900578E0FEA3E0FFC394F7C9
:101BE000EE6480947F7BFF50067A3279FA80047A23
:101BF0003279FD900511EBF0A3EAF0A3E9F0A3EE32
:101C0000F0A3EFF0A37401F0FB7A057967121E765A
:101C10007E337F5A7D05123C659005537401F0A315
:101C20007405F0A3744FF0021DF790050B74FFF0DC
:101C3000A37433F0A37401F090054EE075F005A491
:101C40002444F582E43403F583E0FE3395E0900507
:101C50000EF0A3CEF0A37401F0FB7A057967121E93
:101C6000767E337F737D04123C659005537401F0DA
:101C7000A37405F0A37450F0021DF790054EE075B3
:101C8000F005A42440F582E43403F583E02401FF49
:101C9000EF641190050B6003021D4E74FFF0A374F6
:101CA00033F0A37414F090054EE02434F8E6900568
:101CB0000EF07B017A057956121E7690050B74FFA3
:101CC000F0A37433F0A37426F090054EE0FF75F096
:101CD00005A42441F582E43403F583E0FEC4540FE7
:101CE0002401FCE43390050EF0A3CCF0EE540F2455
:101CF0002AF8E6FC3395E0A3F0A3CCF0EF75F005ED
:101D0000A42442F582E43403F583E0FFC4540F2495
:101D100001FCE433900512F0A3CCF0EF540F242A19
:101D2000F8E6FE3395E0A3F0A3CEF07B017A0579C7
:101D300067121E767E337F967D05123C65900553B3
:101D40007401F0A37405F0A37452F0021DF774FF40
:101D5000F0A37433F0A3743DF090054EE0FF2434FB
:101D6000F8E690050EF0EF75F005A42440F582E446
:101D70003403F583E02401FFE43390050FE4F0A37E
:101D8000EFF07B017A057956121E7690050B74FFF1
:101D9000F0A37433F0A37450F07B017A05796712D5
:101DA0001E7690054EE075F005A42441F582E434DA
:101DB00003F583E0FD7B017A05797012408B900575
:101DC0004EE075F005A42442F582E43403F583E087
:101DD000FD7B017A05797412408B900573743AF09B
:101DE0007E337F877D03123C659005537401F0A319
:101DF0007405F0A37451F09006727401F0A3740599
:101E0000F0A37467F07B017A0579561246E8024127
:011E1000C60B
:03000000020A00F1
:03000300021A03DB
:03000B00021A06D0
:03001300021A09C5
:03001B00021A0CBA
:03002300021A0FAF
:03002B00021A12A4
:03003300021A1599
:03003B00021A188E
:03004300021A1B83
:03004B00021A1E78
:03005300021A216D
:03005B00021A2462
:03006300021A2757
:03006B00021A2A4C
:03007300021A2D41
:100A0000E4F5D9E5EF7480F5FF7402F5EF787FE443
:100A1000F6D8FD9000007F007E10E4F0A3DFFCDE3E
:070A2000FA758161020A6210
:100A2700021626E493A3F8E493A34003F68001F2A9
:100A370008DFF48029E493A3F85407240CC8C333D0
:100A4700C4540F4420C8834004F456800146F6DF9F
:100A5700E4800B01020408102040809033AFE47E4D
:100A6700019360BCA3FF543F30E509541FFEE49394
:100A7700A360010ECF54C025E060A840B8E493A35B
:100A8700FAE493A3F8E493A3C8C582C8CAC583CA86
:100A9700F0A3C8C582C8CAC583CADFE9DEE780BE3E
:0134C7000004
:10217600E709F608DFFA8046E709F208DFFA803E4B
:1021860088828C83E709F0A3DFFA8032E309F60838
:10219600DFFA8078E309F208DFFA807088828C83A0
:1021A600E309F0A3DFFA806489828A83E0A3F60854
:1021B600DFFA805889828A83E0A3F208DFFA804C2E
:1021C60080D280FA80C680D4806980F28033801005
:1021D60080A680EA809A80A880DA80E280CA80336E
:1021E60089828A83ECFAE493A3C8C582C8CCC583E6
:1021F600CCF0A3C8C582C8CCC583CCDFE9DEE780B6
:102206000D89828A83E493A3F608DFF9ECFAA9F034
:10221600EDFB2289828A83ECFAE0A3C8C582C8CC8A
:10222600C583CCF0A3C8C582C8CCC583CCDFEADEA3
:10223600E880DB89828A83E493A3F208DFF980CC05
:1022460088F0EF60010E4E60C388F0ED2402B404FE
:102256000050B9F582EB2402B4040050AF232345A5
:0622660082239021C673E3
:10226C00BB010689828A83E0225002E722BBFE0270
:09227C00E32289828A83E49322A3
:10228500BB010CE58229F582E5833AF583E022500E
:1022950006E92582F8E622BBFE06E92582F8E22258
:0D22A500E58229F582E5833AF583E4932272
:1022B200BB010989828A83F8E028F022500327F7BC
:1022C20022BBFE05F8E328F3228A838982F8E4938D
:0222D2002822C0
:1022D400BB010689828A83F0225002F722BBFE01E9
:0222E400F322E3
:1022E600F8BB010DE58229F582E5833AF583E8F02E
:1022F600225006E92582C8F622BBFE05E92582C8DA
:02230600F222C1
:10230800BC000BBE0029EF8DF084FFADF022E4CCB9
:10231800F875F008EF2FFFEE33FEEC33FCEE9DEC82
:10232800984005FCEE9DFE0FD5F0E9E4CEFD22EDC8
:10233800F8F5F0EE8420D21CFEADF075F008EF2F12
:10234800FFED33FD4007985006D5F0F222C398FD03
:052358000FD5F0EA22A0
:10235D00C2D5EC30E709B2D5E4C39DFDE49CFCEE9B
:10236D0030E715B2D5E4C39FFFE49EFE122308C3E8
:10237D00E49DFDE49CFC800312230830D507C3E4E3
:06238D009FFFE49EFE220A
:10239300C5F0F8A3E028F0C5F0F8E58215827002D5
:0623A3001583E038F02272
:1023A900A3F8E0C5F025F0F0E582158270021583E7
:0623B900E0C838F0E82244
:1023BF00EB9FF5F0EA9E42F0E99D42F0E89C45F074
:0123CF0022EB
:1023D0007401FF3395E0FEFDFCA3A3A3E0CF2FF033
:1023E000E582158270021583E0CE3EF0E58215820B
:1023F00070021583E0CD3DF0E582158270021583F1
:05240000E0CC3CF022DD
:10240500A8828583F0D083D08212241C12241C124A
:10241500241C12241CE473E493A3C583C5F0C5836F
:10242500C8C582C8F0A3C583C5F0C583C8C582C821
:012435002284
:10243600D083D082F8E4937012740193700DA3A335
:1024460093F8740193F5828883E473740293686049
:06245600EFA3A3A380DF49
:06245C008A838982E4730B
:101E1100E51A240BF582E43405F583E0051A2290D6
:101E2100050830070390050BE475F00112248E02BA
:101E3100226C2000E97F2ED2008018EF540F2490ED
:101E4100D43440D4FF30040BEF24BFB41A00500344
:101E51002461FFE51B6002151B051EE51E700205CE
:101E61001D30070E900508E475F00112248EEF0273
:101E710022D402497A7403D2078003E4C207F51A17
:101E81009005081224A5E4F51BF51DF51EE51B6060
:101E9100077F20121E5480F5751CFFC201C200C2CB
:101EA10002C203C205C206C208121E20FF700D3015
:101EB10007057F00121E65AF1EAE1D22B4255FC24D
:101EC100D5C204121E20FF24D0B40A00501A75F0A6
:101ED1000A781B30D50508B6FF0106C6A426F620F0
:101EE100D5047002D20380D924CFB41A00EF500474
:101EF100C2E5D204022066D20180C6D20080C0D2DF
:101F01000280BCD2D580BAD20580B47F20121E5483
:101F11002002077401B51B0040F1121E11FF121EB1
:101F210054021E8ED208D2068095121E11FB121E7B
:101F310011FA121E11F94A4B700679377A217BFF8B
:101F410020022EE51B602A7E008E827583001222FC
:101F51008560060EEE651C70F0C2D5EBC0E0EAC0EC
:101F6100E0E9C0E0EE1220ADD0E0F9D0E0FAD0E037
:101F7100FB12226CFF60AAEBC0E0EAC0E0E9C0E01E
:101F8100121E54D0E02401F9D0E03400FAD0E0FB75
:101F9100E51C0460DCD51CD980877BFF7A2079A9F8
:101FA100D202809C791080027908C206C20880089A
:101FB100D2D5790A8004790AC2D5E51C047002F5EC
:101FC1001CE4FAFDFEFF121E11FC7B082001131216
:101FD1001E11FD7B1030000A121E11FE121E11FF90
:101FE1007B20EC3382D592D55013C3E43000069F99
:101FF100FFE49EFEE42001039DFDE49CFCE4CBF89C
:10200100C201EC700CCFCECDCCE824F8F870F3808F
:1020110017C3EF33FFEE33FEED33FDEC33FCEB334F
:10202100FB994002FB0FD8E9EB300105F8D0E0C481
:1020310048B201C0E00AEC4D4E4F78207B0070C2DF
:10204100EAB51C0040BCC0E01220AFD0F0D0E020C7
:102051000104C4C0E0C4B201C0F0121E3DD0F0D5ED
:10206100F0EB021E8E1224361F2B531FA5581EFCA7
:102071004C1EF8421FA94F1FB1441FB1491F114304
:082081001FB7551F9B461F9B72
:10208900451F9B472157501F002D1F042E1F272B2B
:102099001F08231F252021402A1EC04800001F1F9A
:1020A9003F3F3F00790AA2D5200314300509B91032
:1020B900020404B9080104A2D52006025001042033
:1020C90002689202B51B005034C0E07F203003192A
:1020D9007F30A20272067205500F122106C202C297
:1020E90006C205C2087F30800F300503E9C0E0123F
:1020F9001E54300503D0E0F9D0E0B51BCC300517EC
:102109007F30B9100C121E547F583004077F788035
:1021190003B90803121E543002057F2D021E547F95
:10212900202008F87F2B2006F322920280CF286E08
:10213900756C6C2900D201121E113001F8C20178A8
:102149001B30D50108F6021EC02D50434958121EF6
:10215900112403B405004001E490215293121E4555
:0D216900743A121E45D203751B04021FA517
:10246200EF4E6012EF60010EEDBB010B89828A8391
:10247200F0A3DFFCDEFA2289F05007F709DFFCA99E
:0C248200F022BBFEFCF309DFFCA9F022F5
:10248E00F8E0FBA3A3E0F925F0F0E58215827002D7
:07249E001583E0FA38F0227B
:0924A500EBF0A3EAF0A3E9F02238
:10497A00EFB40A07740D124985740A309811A89980
:10498A00B8130CC2983098FDA899C298B811F6309D
:07499A0099FDC299F5992275
:00000001FF
